:020000040000FA
:2000000018F09FE5FEFFFFEA600000EAFEFFFFEAFEFFFFEAFEFFFFEA660000EAFEFFFFEA3C
:04002000400000009C
:20004000D3F029E30000A0E30110A0E398219FE5001082E594419FE55550A0E3AA60A0E3F8
:20006000082094E5020412E3001084150C6084150C508415000084E50C6084E50C5084E53E
:200080006C219FE5000082E50128A0E3472082E3042084E50C6084E50C5084E5001084E5D0
:2000A0000C6084E50C5084E5082094E5010312E3FCFFFF0A3C219FE50330A0E3003082E5DA
:2000C0000330A0E3003084E50C6084E50C5084E524219FE5000082E5040082E51C119FE5EB
:2000E000D7F029E301D0A0E1041041E2DBF029E301D0A0E1041041E2D1F029E301D0A0E125
:20010000101041E2D2F029E301D0A0E1021B41E2D3F029E301D0A0E1E4809FE5E4909FE53B
:20012000E4A09FE509A05AE00300000A0100B8E80100A9E804A05AE2FBFFFF1ACC909FE5C1
:20014000CCA09FE509A05AE00300000A0000A0E30100A9E804A05AE2FCFFFF1A0151A0E3E1
:20016000050059E10950A081A8C09FE500508CE588509FE5A0C09FE500508CE59CC09FE538
:200180000000A0E30FE0A0E11CFF2FE1FEFFFFEA04E02DE504C02DE500C04FE104C02DE5C9
:2001A00004C01EE5FFC4CCE374E09FE50CC18EE000E09CE51EFF2FE104E04EE200402DE9FB
:2001C00000102DE900C04FE100102DE908002DE9FFE0E0E300E09EE544C09FE50EC18CE0FD
:2001E00000309CE50FE0A0E113FF2FE140C01FE080C01FE00CC11FE004C11FE0A8C11FE086
:2002000000000140302600000000004030000040B8280040CC280040C4280040C8280040E7
:20022000C9020000300000407047C0467047C04600B5054800F018F90120404200F000F97A
:20024000002002BC0847C0466024000000B5034800F00AF9FFF7ECFF02BC084718240000CA
:20026000002070470020704700B5431C0FD0C31C17D0831C08D00E4A031C1340934203D02E
:200280001120404202BC084709204042FAE7094800F0EAF80120404200F00EF9292040428A
:2002A000F0E7054800F0E0F809204042EAE7C046000000FF90240000A824000000B500F0AC
:2002C00071F8002002BC084700B500F03BF8034800F034F9002002BC0847C0463C240000B5
:2002E00000B500F01BF8FFF7B1FF00F003F801BC0047C04610B5041CFFF7B4FF002C07DB0F
:20030000054800F0B1F800F0FDF810BC01BC0047201CFFF7A9FFF6E7C024000000B500F002
:20032000A3FE002805DBFFF79BFF002801DB01BC0047034800F098F800F080F8F7E7C04665
:20034000D824000000B5FFF7B9FF002805DB00F0EFFF002801DB01BC0047034800F084F899
:2003600000F06CF8F7E7C046F024000010B50C1C002910DD0021094B1B689A06FBD502784C
:20038000074B01311A60A14201D00130F3E7201C10BC02BC08470020FAE7C04614C000E0D0
:2003A00000C000E010B511490B68082213430B600F490B68F0229343502213430B600D4CE1
:2003C0000D490020802308602360FF230B600B4B1D221A6003221033086022601A60072288
:2003E000083B1A6010BC01BC0047C046C4C01FE000C002E00CC000E004C000E000C000E055
:2004000030B50D1C002913DD00240A4B1A68D306FBD0094B19681E231A42F6D10134017037
:20042000AC4201D00130F0E7281C30BC02BC08470020FAE714C000E000C000E0FEE7C04678
:2004400030B581B002F0E0F86C460334051C0121201CFFF7D5FF281C02F0DAF8207801B039
:2004600030BC02BC0847C04630B5041C02F0CCF82378051C002B08D115E0201C012101347A
:20048000FFF774FF2378002B0DD00A2BF5D109480121FFF76BFF201C01210134FFF766FF94
:2004A0002378002BF1D1281C02F0B2F8002030BC02BC08475C240000FEE7C04600000FE160
:2004C000C0C080E30CF021E11EFF2FE1C03000E200000FE1C020C0E3032082E102F021E14F
:2004E0001EFF2FE100F021E11EFF2FE100000FE11EFF2FE100B500F095F900F019FA01BCA0
:200500000047C04600B5FFF7F5FF00F0DFF901BC0047C04610B50C1C00F0A6F8002802DB9D
:2005200010BC01BC0047201CFFF79EFF0248FFF79BFFFFF783FFF3E70825000010B5041CDE
:2005400002F062F828492948FFF7E4FF28492948FFF7E0FF28492948FFF7DCFF2849294848
:20056000FFF7D8FF28492948FFF7D4FF28492948FFF7D0FF28492948FFF7CCFF28492948D7
:20058000FFF7C8FF28492948FFF7C4FF28492948FFF7C0FF28492948FFF7BCFF28492948F7
:2005A000FFF7B8FF28492948FFF7B4FF28492948FFF7B0FF28482949FFF7ACFF201C00F0CD
:2005C00021FB002809DB002100F09AFB002804DB234B184710BC01BC00472248FFF744FF06
:2005E000FFF72CFFF4E7C046242500001D09000028250000E108000030250000FD100000F2
:2006000038250000AD0F0000442500004D0E000050250000850E000058250000190F000050
:2006200068250000790F000074250000510F000080250000F10E00007C250000B90E0000A0
:200640008C250000E50F00009C25000019100000AC2500005110000031080000B8250000C3
:2006600034090000C02500000047C046F0B5144D2A6882B08446AA4216D0C1688068936899
:20068000D468061C0F1CF61AA74100960197002F0ADB1268AA4207D09368D468061C0F1CD6
:2006A000F61AA741002FF4DA536867467B60536802B03A6057601F60F0BC01BC0047C0460F
:2006C0000402004030B50D1C026143614B1C11D00A4B19685A680A230024C91862412B1CC3
:2006E000EC17C91862418160C260FFF7BFFF30BC01BC004700604060F9E7C046F4010040B1
:20070000F0B543610B4B1D685E6802610A220023521973410C1C0025161C1F1C36196F4165
:20072000331C3C1C8360C460FFF7A0FFF0BC01BC0047C046F401004000B50361019B8160F5
:20074000C2604361FFF792FF01BC0047F0B52B4B10221A602A4BFF221A60122001F05CFFF3
:2007600001F052FF274E336874680A2100225B18544133607460244D071C2868A84207D0AA
:200780008168C26833687468C91AA241002A1FDDC0231F420DD11D4B1D4A1968136899421B
:2007A00007D01C4B1B68002B03DC1B4B1B68002B20D0381C01F02CFFD22001F02DFF174B89
:2007C00000221A60164B10221A60F0BC01BC0047002A01D10029DBD80368834203D042683B
:2007E000136003685A600369002BC6D0406900F06BF8C2E701F014FFDBE7C04614F0FFFFC1
:20080000004000E0F401004004020040B8110040BC110040B8280040B411004000FFFFFF05
:2008200010F0FFFF00B5042001F076FB01BC004710B51C4A00230024136054601A4A13600B
:2008400054601A4B1B605B6001F0DEFE18490B68022213430B60174C174B002222601A60E0
:20086000343B1A60143B1A6014491C3B1A600C331960083B1A60083B1A60FF22083B1A6088
:20088000032214331A600123236001F0C1FE0C4A0C4B04201361052101F022FB002010BCB6
:2008A00002BC0847FC010040F401004004020040C4C01FE0044000E0704000E01FBF02005C
:2008C00030000040B40B00001847C04600B501F09BFE0020FFF7F0FDFFF7B0FDFCE7C046B6
:2008E0000A4A01235B42136008321360084B0021084A196018331A60DC33074A19600123C2
:2009000008C20133202BFBD10020704714F0FFFF0CF0FFFFFFFF000004F1FFFF0249034A66
:2009200090230020CA50704730000040440B00007047C046A4D29FE5A4C29FE50100A0E32F
:2009400000008CE59C429FE50000A0E3000084E513F021E3110000EA00502DE900C00FE1C0
:20096000C0C0CCE300102DE900402DE970C29FE501E0A0E300E08CE513F021E368C29FE5AC
:2009800000C09CE53CD04DE2FF7FCDE854429FE50000A0E3008094E570D088E5000084E5FC
:2009A00048529FE548629FE5D3F021E3008095E5000058E30400001A00C096E500005CE357
:2009C0000707000B13F021E3F6FFFFEA008084E570D098E508C29FE500E0A0E300E08CE571
:2009E000FF7FDDE80000A0E13CD08DE2F8E19FE500C08EE50040BDE80010BDE80CF06FE142
:200A00000090FDE808002DE9030000EA00E00FE11FE00EE213005EE308002D0907002DE9E8
:200A2000D0319FE503304CE02301A0E110108DE200200FE1D2F021E304402DE900102DE948
:200A4000B4C19FE500E09CE501E08EE200E08CE5A8C19FE503C09CE70FE0A0E11CFF2FE1CC
:200A60000010BDE80C00BDE8C02082E302F021E184C19FE500E09CE501E04EE200E08CE54B
:200A80000700BDE893300DE1FFFFFFEB00C00FE11FE00CE213005EE31100000AD3F029E336
:200AA00070002DE900402DE904002DE904208DE20CF029E1C0C08CE320C0CCE311005EE3D7
:200AC0000CF021E10050BDE804E082E50050BDE808C082150CE082E5D3F021E30400BDE8C1
:200AE000000000EAD3F021E30CC19FE500C09CE500005CE30C00001AE4C09FE500C09CE5E5
:200B000000005CE30800001A04C09DE5C0001CE30500001ACCC09FE5D0E09FE500C09CE5CB
:200B200000E09EE50E005CE18FFFFF1A0040BDE80010BDE80CF06FE10090FDE80900E0E339
:200B40001EFF2FE100005CE3020000AA00502DE900C00FE100102DE9000C2DE908B08DE2F8
:200B600084C09FE500A09CE500042DE90AE8A0E100E08CE504E09BE500005EE3090000AA56
:200B8000060000EA0CD04BE2020CBDE858C09FE500108CE50010BDE80CF06FE10090FDE816
:200BA0000900E0E3F7FFFFEA0E10A0E18F0600EBF4FFFFEAD2F021E337402DE938409FE540
:200BC000005094E5010085E2000084E58A0600EB005084E53740BDE89E300DE1AAFFFFEBDC
:200BE0008C020040B4110040B8110040F0010040BC110040BC28004030000040B828004027
:200C00008C020040F0B5474680B44268354B051C1A4207D00B246442201C04BC9046F0BCCF
:200C200002BC0847C368013B1F2B02D911246442F2E701697F29F9DDCB1DDB10DE00930635
:200C400041D5B142F2D1C76901F0DEFC264A14688046944240D02368136023685A602B685F
:200C6000224AE3606B6813402361AB686361EB682022013BA354BB19E3660123A66123779A
:200C8000E383201C00F084FAA468C02342461A420DD1174B174A19681368994207D0164BC1
:200CA0001B68002B03DC154B1B68002B17D0404601F0AEFC002CAFDA6B689A06ACD4381C95
:200CC00000F006FBA8E7301C00F0C0FA071C0028BAD1212464429FE722246442D5E701F0BE
:200CE0009FFCE4E7DEFCFFFF50210040FFFCFFFFB8110040BC110040B8280040B4110040D1
:200D0000F0B52B4E33680F1C0022002B2CDD0122431E1F2B34D8002A03D1264B1B68002BA2
:200D200038D174224243244B743BD41801F06CFC2323E35C051C082B30D0002B1DD02924EE
:200D40006442C0231D4208D11A4B1C4A19681368994202D03368002B15DD281C01F058FC1D
:200D6000201CF0BC02BC0847124B1B68002BCFD00028CDD129246442F2E72A246442E0E787
:200D800012246442ECE70E4B1B68002BE5D101F047FCE2E79B688342C3D1EBE7226FE368E0
:200DA000201C1760536000F023FA0024C9E7C046B8280040B8110040D0120040BC1100408E
:200DC000B4110040F0B5FF230A1C1A40531E071C0C1C032B2ED8194B9200043BD618184B51
:200DE0001B68002B1FDC174D2B68002B1BD001F00BFC2A68D38B0133D383002001F008FCB6
:200E00003368211C381C00F01FF8041C01F0FCFB2A68D38B013BD383002001F0F9FB201CD4
:200E2000F0BC02BC0847211C3368381C00F00CF8041CF4E70A246442F1E7C046440F004099
:200E4000B8280040B81100401847C04610B50B490B4C0960496000200219002393604B687E
:200E6000116053601A60C02318305B004A609842F2D1002010BC02BC0847C046CC050040F7
:200E80004C04004010B50A490A4C096049600020031900229A604A681C305A6019604B600E
:200EA0001360E028F4D1002010BC02BC0847C046B4060040D405004010B50B490B4C096007
:200EC00049600020031900221A639A604A6819605A6013604B60E02338305B009842F1D12F
:200EE000002010BC02BC08477C080040BC060040074B002207499A60DA631A1C343200207C
:200F00000B6059609B6359631A604A607047C04684080040EC08004010B50B490B4C096039
:200F2000496000200219002393604B68116053601A60D02334305B004A609842F2D100204D
:200F400010BC02BC0847C046940A0040F4080040074B002207499A609A621A1C2032002036
:200F60000B6059605B6219621A604A607047C0469C0A0040DC0A004010B50A490A4C096051
:200F800049600020031900229A604A6824305A6019604B6013609028F4D1002010BC02BCD2
:200FA0000847C046740B0040E40A004010B50B490B4C0960496000200219002393604B6869
:200FC000116053601A60E0231C305B004A609842F2D1002010BC02BC0847C0463C0D0040FA
:200FE0007C0B004010B50A490A4C096049600020031900229A604A682C305A6019604B6066
:201000001360B028F4D1002010BC02BC0847C046F40D0040440D004010B50B490B4C096016
:20102000496000200219002393604B68116053601A60A02328305B004A609842F2D1002088
:2010400010BC02BC0847C0463C0F0040FC0D0040034A044B0020136053609360D36070471E
:20106000440F00403C0B000030B51649164800F09BFF041C002822DB144B1549154A1B608E
:201080005B6009604960101C4B6890240025A400536011604A601A601572031948329A42E6
:2010A000F2D100F0D1F9041C002808DB0A4B1D6000F080F90024201C30BC02BC084700F004
:2010C0000DF8F8E7DC250000A4110040941100409C110040540F0040B011004010B500F00B
:2010E0007FF900F0E7F9041C034800F079FF201C10BC02BC0847C046A411004070B51E4B37
:2011000000221A601D4B1E481A60202303600021CA00131D1B1812180131536093602029AC
:20112000F6D1822300245B00C45086235B00C45084235B00C0180021042200F037FE114BF6
:201140001C60114C114E2460646000230025581CAB19191C002223310A7062681C605A606A
:2011600098605866136063607435031C2028EED1002070BC02BC0847BC110040B811004045
:20118000C0110040B411004050210040D012004030B508222323C2542023C25C2123C25440
:2011A0002223C2541C23C356051CC38300202863686324216B5C0124A3436B546B5C0222DE
:2011C00093436B54EB6E69691A1CA863A8664C3A21420AD03320002313630123994391645C
:2011E00010642A6730BC01BC00471320F3E7C04670B501222323C2542223C65C114C721CF1
:20120000D20013594360F30004331B19036013591051842252001860051C311CA01800F0D9
:20122000FDFD2423EB5C9A0702D586235B00E55023689E4202DA044B26601D6070BC01BCF3
:201240000047C046C0110040BC110040F0B557464646C0B40F2826D810229046102401F07F
:20126000D3F91A4F8246211C386800F055FA3B680C33051C984226D000F0A4FAEB68424619
:201280002E1C9B1A083E172B13D87368012213437360504601F0BCF9281C0CBC90469A46B7
:2012A000F0BC02BC0847C21D07239A439046141CD5E7AC18301C211C00F0A6FA3868211C13
:2012C00000F052FAE1E70025E3E7C046B4280040F0B5041C01F098F9251C083D6C68012631
:2012E000B443071C6C6028684368334215D06368334207D1201C083000F064FA206800F021
:2013000091FA251C094B291C186800F02DFA381C01F07EF9F0BC01BC0047083000F052FAF1
:20132000286800F07FFA6C68E1E7C046B4280040F0B51B4B1F681B4B3C1C9F422CD81A495E
:201340000B680722073393431D1C1435641B181C103C164E10C01A1C2C190C3208343360A4
:201360000F6058609860DA601A61211C00F04CFA3068291C043000F047FA636801221343A0
:2013800030686360836813438360291C00F0ECF90020F0BC02BC0847054F3C1CCFE7C04673
:2013A000C8280040FFFF0040C4280040B42800400000014010B5084C0021201C00F0D4FDFF
:2013C000064B00221B605B609A60201C002100F0D3FD10BC01BC0047A4110040A828004078
:2013E00070B5164D2B68002B24D0154E0021301C00F0BAFD1349AA680B682C689B1A0B60A7
:201400000023AB60AC4211D00023083C23610021301C00F0B1FD201C002100F04DF8301CFB
:20142000002100F0A1FD2C68AC42EDD1301C002100F0A2FD70BC01BC0047C046A82800407B
:20144000A4110040C028004070B51648164E0060406000240025AA19002341681361A30198
:201460009B1901345160106043600B604035102CF1D10E480E4E0060406000240025AA1923
:20148000002393603423634341689B1901345160106043600B603435102CF0D1002070BCC6
:2014A00002BC08475825004058210040A02800406025004000207047F0B55F4656464D468C
:2014C0004446F0B48F4F81B0061C0091381C002100F04AFD73699A6B92465A6B5B69934655
:2014E000994600F0ADF90023B363336B7063002B00DCD6E0F46A01F087F8834D2A68D38B82
:201500000133D383103C002001F082F8F16A326B4B46E06800F0FEF801F076F82A68D38B64
:20152000013BD383002001F073F8B36B0133B36320239B199846381C002100F01DFDB36BC3
:20154000002B05DD0122F06B0121524200F002FA00237363381C002100F006FD346A4445D6
:201560002ED001235A42684D9246237F1022134323770021381C00F0FFFC01F045F82A683C
:20158000D38B0133D383002001F042F8201C012152464B46103000F0BEF801F035F82A68FB
:2015A000D38B013BD383002001F032F80021381C00F0DAFC201C00F081FA346A4445D4D152
:2015C0000021381C00F0D8FC0021381C00F0CCFC7569B369EA6A98466B69F06B9246994693
:2015E00000F036F9301C002100F046FA281C414600F078FA002806D0AB69012213424AD05E
:20160000009B93430093381C002100F0B5FC5246002A44D000F0F8FF3B4C2268D38B013350
:20162000D383002000F0F4FF384AAA1AD210D3009B1A99015B18DB009B18D803C01AC00091
:201640008018013000024A460099404400F062F8051C00F0D9FF2268D38B013BD383002045
:2016600000F0D6FF381C002100F07EFC284B5A6872605A6833605E601660381C002100F0D1
:201680007BFC281C01B03CBC90469946A246AB46F0BC02BC0847381C002100F06DFC0025AC
:2016A000E0E720229219346A9046444504D142E72468444500D13EE7E368002BF8D0237F90
:2016C00010221343237700F09FFF0F4D2A68D38B0133D383002000F09BFF211C1031012239
:2016E0004B46E06800F016F800F08EFF2A68D38B013BD383002000F08BFFB36B0133B36312
:20170000D6E7C046A4110040B8110040540F0040582500405047584710B50368021C041C04
:201720000C32002B1DDB9B108B4209DB101C0068824214D0C3689942F9DC10BC02BC0847FC
:20174000101C00234068824206D0C3689942F9DB9942F2DD0068F0E7994200DCE268101C08
:20176000EBE70333DFE7C046F0B50B680E1C08369F1B0D1C391C041CFFF7CEFF6B68012204
:2017800093430C346B60A04204D0011C08314B68BB420BD043687360436830601E60002377
:2017A00046602B616F61F0BC01BC004783682A1C10322B6182602B6951605A600023AB6069
:2017C000F1E7C0460368002B16D08268011C0831002A0AD04368083A53604368106042600E
:2017E0001A604B68826853600368984203D04268136003685A607047C2688368136080689E
:201800000028F8D04260F6E710B503680B60486004686368012213400B436360016010BC2B
:2018200001BC004710B5426801240368A243136001684B6823401A434A6010BC01BC0047F7
:20184000024B1868002800D080687047B811004030B5431E0F2B05D912246442201C30BCB9
:2018600002BC0847194BC200121A1C3B9200D41800F0CAFEA368051C002B16D12A2464424A
:20188000C0231D420DD1124B124A19681368994207D0114B1B68002B03DC104B1B68002BCF
:2018A00011D0281C00F0B4FED8E7201C00F04CF90B4A53686360536822601C6000235460CE
:2018C000A3600024DCE700F0ABFEEAE77C0B0040B8110040BC110040B8280040B4110040B2
:2018E0003C0D004070B5041CE26A1548D3009B1A1C389B001E18002903DB301C211C00F044
:201900008BF933699A0717D43068B04214D07269C36B041C05689A4205DA0DE02C1CE36BD9
:201920002D68834208DC201C00F0ECF87269E36BD01A7061AE42F1D170BC01BC0047C0468D
:201940007C0B004000B501214942FFF7CBFF01BC0047C046F0B557464E464546E0B4431E3E
:2019600081B0041C0D1C161C0F2B09D91220404201B01CBC90469946A246F0BC02BC08470C
:20198000002902DC11204042F2E7511CFADB334A92461268002A02D019204042E8E7304BA2
:2019A00099461B68002BF7DC2E4F3B68002BF3D0009200F039FEC0231842EDD12A4BE200AE
:2019C000121B1C3B9200D41800F01EFEA3688046002B1AD12A235B420093C02342461A42CE
:2019E0000ED1224B3A681B689A4209D049460B68002B05DC52461368002B01D100F010FEA5
:201A0000404600F005FE0098B2E7A3699D4203DD11235B420093E0E72369990705D5636954
:201A20009D4209DC5B1B6361D7E73968201C00F015F93B689842F2D023693A68D9070AD5E3
:201A40000B4B93623A686B469363D563201C311C00F0AAF8C1E7074BF3E7C046B4110040C0
:201A6000B8280040B81100407C0B0040BC110040000000400C00004010B503680C1C8342C0
:201A800003D04268136003685A60031C81680833994203D0C268116083685A60002C06D0FE
:201AA000054B5A6842605A680360586010600023036110BC01BC00475825004003688342E1
:201AC00003D04268136003685A60054A536843605368026018600023506083607047C0463C
:201AE000A0280040026C4030824203D107E01268824204D093698B42F9D1012000E00020BB
:201B00007047C04610B5031CC16C4C33041C994203D0026D1160C36C5A602368A34203D09E
:201B20006268136023685A602322A35C022B07D00423A354A26B0023136010BC01BC00474A
:201B4000201CFFF755FBF5E730B50468051CA04209D126E00423A354A26B33232C685B4241
:201B60001360A5421DD0231CE16C4C33994203D0226D1160E36C5A602368A34203D062684F
:201B8000136023685A602322A35C022BE2D1201CFFF72EFBA26B33232C685B421360A54220
:201BA000E1D130BC01BC004730B51A4D041C081C296832238A6B5B421360002802D130BC21
:201BC00001BC0047A368CB62216900F05BF82369DA0716D52D6822682223201CE95C9442E9
:201BE00004D107E01268944204D02223D35C8B42F8D9101C43686B604368286045601D60FC
:201C0000DDE72B6862685A6062681C6063601360D5E7C046B811004030B50B680C1C051C01
:201C2000A34203D04A6813600B685A602A682223291CE05C954204D107E01268954204D08A
:201C40002223D35C8342F8D9111C4B6863604B6821604C601C6030BC01BC004710B50C1C9E
:201C60000168814207D00369DA0708D52223E25CCB5C9A4203D2201C10BC02BC08470C1C9F
:201C8000F9E7C04670B50D4C061C20682325435D012B0DD0042B01D1062343552368181CC4
:201CA000311C074A4C30FEF70DFD70BC01BC004700F008F8226802235355EFE7B8110040B5
:201CC000711D0000F0B5474680B4274D862222235200C65CAB58041C984240D02368A342BE
:201CE00003D06268136023685A602421635C012213420AD0934363541C4A1368A34221D0F5
:201D000004BC9046F0BC01BC0047F3005A19526804335B199A42EFD184235B005B19181C6C
:201D2000311C984600F088F82F68B742E4D12026F21B4046391C00F08DF8002812DBC3192F
:201D40002B60D9E786235B00EB58002B01D01360D6E72B68DB005B195B681360D0E70023D3
:201D6000AB50BBE72E60C7E7C0110040BC11004010B50368041CA34203D0426813600368DC
:201D80005A602322A35C022B0BD00423A354A36A9B68002B02D0201C00F007F810BC01BC5E
:201DA0000047201CFFF724FAF1E7184730B5051C0906101C2B1C090E072A0AD8002A04D0A5
:201DC0000023595501338342FBD1281C30BC02BC0847AA071AD01970013301389A07FAD133
:201DE0000A041C1C0B0213430B430A061343032803D9043808C40328FBD80028E5D0231C5D
:201E00000138197001330028FAD1DEE70A040B0213430B430A062C1C1343EAE70A1C002987
:201E200008DBC91007231340091801229A400B7813430B707047C0460A1C002908DBC9102F
:201E400007231340091801229A400B7893430B707047C04630B5141C002904DA0120404297
:201E600030BC02BC0847002AF8DB002AF6D0CB101D180A1C07231A4080235B0493402A784B
:201E80001B0E002A11D1002006E00830A042E5DA01352A78002A09D10028F6D107230A1C13
:201EA0001A400823981A0123F0E700201A4204D15B061B0E01301342FAD08442D0DCCDE79F
:201EC0001F2809D8054B1A6801238340181C104000D170470120FCE70020FAE708F0FFFF1A
:201EE00030B5051C0C1C00F08FFB064AAB009B181C60054A0123AB40136000F089FB30BCDF
:201F000001BC004700F2FFFF10F0FFFF014B00221A60704700FFFFFF024A0123834013608D
:201F20007047C04614F0FFFF30B5041C00F06CFB0B490B680B4A1D1C10231B1B15401A4118
:201F40000A6000F065FB002D07D000206D080130002DFBD130BC02BC08470020FAE7C04604
:201F600024F0FFFFFFFF000000B50122524200F049F802BC0847C04630B50123041C1D1C3F
:201F80008D4000F041FB2368AB43236000F040FB6368002B03D1002030BC02BC0847A06836
:201FA000291C00F0FFF8F7E770B585B0051C002914D06846042200F015FA092300246846BE
:201FC0000193029400F04EF8A860002802DB6C602C60002005B070BC02BC08470091ECE7CA
:201FE00010B5041C8068002809DD00F091F8002802DB0023A360002010BC02BC0847112038
:202000004042F9E7F0B50123051C1E1C82B0171C8E4000F0F9FA6B6801336B6000F0F8FA70
:2020200000F0F2FA2C68331C23432B6000F0F0FA264215D0A868311C212201AB009700F0F6
:202040002BF9041C0028EBDA00F0DEFA6B68013B6B6000F0DDFA201C02B0F0BC02BC08473F
:202060000024F1E730B542680923041C9A4305D00B246442201C30BC02BC084700F0C4FA1F
:202080001D4A051C1068904230D00368136003685A601A4A821AD21093009B1819015B18B6
:2020A00019025B1819045B185B009B18226801338360C26062680261A26800604060426157
:2020C0001C1CC0231D420DD10D4B0E4A19681368994207D00C4B1B68002B03DC0B4B1B688D
:2020E000002B06D0281C00F093FAC3E722246442E7E700F095FAF5E7CC0500404C040040BE
:20210000B8110040BC110040B8280040B411004030B5431E0F2B05D912246442201C30BC22
:2021200002BC0847194B42001218183BD200D41800F06AFAA368051C002B16D12A2464422B
:20214000C0231D420DD1124B124A19681368994207D0114B1B68002B03DC104B1B68002B06
:2021600011D0281C00F054FAD8E7201CFFF7ECFC0B4A53686360536822601C6000235460C0
:20218000A3600024DCE700F04BFAEAE74C040040B8110040BC110040B8280040B411004084
:2021A000CC050040F0B5474680B4431E0C1C0F2B07D912246442201C04BC9046F0BC02BCED
:2021C0000847284B42001218183BD200D71800F01BFABB688046002B17D12A246442C023E5
:2021E00042461A420DD1204B204A19681368994207D01F4B1B68002B03DC1E4B1B68002B8C
:202200002CD0404600F004FAD5E77B6923437B613D68AF4220D0281C066C2D68C46BF20773
:2022200013D57A692242F4D0436C1A60FFF76AFCB30604D57B69A3437B61002B0CD0F206EF
:20224000E7D5002300247B61C9E77A69131C23409C42E9D0AF42DED10024C0E700F0E0F9AF
:20226000CFE7C0464C040040B8110040BC110040B8280040B411004000B5C36A011C054A89
:202280005800C018183AC0008018FFF7C5FC01BC0047C0464C040040F0B55F4656464D469A
:2022A0004446F0B41F1C431E81B0041C0D1C161C0F2B0AD91220404201B03CBC9046994679
:2022C000A246AB46F0BC02BC0847002902D111204042F1E73123111C9943F8D10A9A0132E8
:2022E000F5DB394B1A689946002A02D019204042E2E736490B688B46002BF7DC344B98468B
:202300001B68002BF2D0009200F08EF9C0231842ECD1304B62001219183BD200D41800F041
:2023200073F9A3688246002B1BD12A235B420093C02352461A420FD1274B41460A681B6825
:202340009A4209D05A461368002B05DC49460B68002B01D100F064F9504600F059F90098E5
:20236000AAE721690A0706D42368A34203D029235B420093DCE7F30714D56269154216D1E9
:2023800043461A68CB071DD5144B414693620B686A46DD631E645F649A63201C0A99FFF719
:2023A00003FCC5E762692B1C13409D42E8D13A60B10602D56369AB436361F206B8D5002327
:2023C0006361B5E7064BE0E7B4110040B8280040B81100404C040040BC1100401800004062
:2023E0002400004010B5041C081C211C00E00130013A0CD303780B7003780131002BF6D173
:20240000013A04D300230B700131013AFAD2201C10BC02BC0847C0460A6D6963726F205420
:202420002D4B65726E656C2056657273696F6E20312E30312E30300A0A0000000000000086
:2024400001000000E10200001E00000000040000696E697474736B00000000000D00000063
:202460005075736820616E79206B657920746F2073687574646F776E20746865206D696392
:20248000726F20542D4B65726E656C2E0A0000000A3C3C2053595354454D205245535441FB
:2024A0005254203E3E0A00000A3C3C2053595354454D205245424F4F54203E3E0A000000B8
:2024C0000A3C3C2053595354454D2053485554444F574E203E3E0A00214552524F52212047
:2024E00073746172745F73797374656D0A000000214552524F522120696E69745F6B65725F
:202500006E656C0A00000000203A206D6F64756C6520696E697469616C697A6520657272B7
:202520006F720A0063707500746B6465760000007461736B0000000073656D6170686F7238
:20254000650000006576656E74666C61670000006D61696C626F78006D6573736167656227
:20256000756666657200000072656E64657A766F757300006D757465780000006669785F15
:202580006D656D6F7279706F6F6C00006379636C696368616E646C6572000000616C6172F3
:2025A0006D68616E646C65720000000073756273797374656D00000074696D6572000000C0
:2025C000696E69745F7461736B2063616E206E6F7420737461727465640A0000444D4C6B09
:2025E0000000000000C09FE51CFF2FE12902000000C09FE51CFF2FE1C50D000000C09FE5BC
:202600001CFF2FE14D0700007847C046AAF7FFEA7847C046ACF7FFEA7847C046B0F7FFEA46
:202620007847C046CBF8FFEA7847C046AEF7FFEA04000000E5180000451900000400000073
:20264000000000004519000008000000792200000000000008000000000000000000000071
:0400000500000040B7
:00000001FF
